:10000000DEFD9E00CEFCBC0000BCD1FFBCD000BC1D
:10001000D9FFBCD800BCD57FBCD47FDD6FBC0E0A35
:10002000313ADEEA9AE89A039AE89E03BDEE7FBC75
:10003000EF11D3FABDEE7C31203159BD047001F9C6
:10004000BD0468318233F2316DED9D0E920E0103D5
:10005000BC0E0ABCD000DED47B7A79789D0E920A61
:1000600068920B69920C6A920D6B9D0E9CFEAE9C81
:10007000D09D0E8A9C0E8E00000000000000000043
:100080000000000000000000000000000000000070
:100090000000000000000000000000000000000060
:1000A0000000000000000000000000000000000050
:1000B0000000000000000000000000000000000040
:1000C0000000000000000000000000000000000030
:1000D0000000000000000000000000000000000020
:1000E0000000000000000000000000000000000010
:1000F0000000000000000000000000000000009C64
:10010000009DFE9C01BDEF6D9DEF9C09304AC3052B
:10011000D3FABD04789D099CEF9D019CFE9D008F44
:10012000BDD47DBDD46CBC07093249BC07773249C8
:10013000BDD47DBDD46CBDD47C8EBDD47DBDD46C0E
:10014000BC07093249BC07353249BC07C03249BD3A
:10015000D47DBDD46CBDD47C8E9DF3937D0FBD0545
:1001600077010ABD0D6DBD0D6EBD0D6F8EBD06779D
:100170000D9D06931D04BD0D7E07BD0D7F03BD0DB6
:100180007D8EBDD47DBDD46CBC07093249BC0755FA
:100190003249BDD47CBDD47DBDD46CBDD46DBC070B
:1001A000893249BDD56CBDD47C31DD9D079C06BD2F
:1001B000D46CBDD57CBDD47DBDD46DBDD56CBDD456
:1001C0007C31DD9D079C05BDD47CBDD57CBDD47D37
:1001D000BDD46DBDD46CBDD47DBDD47C8EBDD47D6D
:1001E000BC0700BDD674BD077FBDD46DB8BDD47D3E
:1001F000BDD674BD077EBDD46DB8BDD47DBDD674EB
:10020000BD077DBDD46DB8BDD47DBDD674BD077CA2
:10021000BDD46DB8BDD47DBDD674BD077BBDD46DD6
:10022000B8BDD47DBDD674BD077ABDD46DB8BDD47C
:100230007DBDD674BD0779BDD46DB8BDD47DBDD6A6
:1002400074BD0778BDD46DB88ED008BDD46D9D0740
:10025000B09C078904BDD47C03BDD46CBDD47DC0E3
:10026000EABDD46DBDD47CBDD47DBDD46DBDD46C90
:100270008E920023E9920123E0920223D792032376
:10028000CE920423C5920523BC920623B392072382
:10029000AA920823A192092398920A238F920B23F2
:1002A00086920C237D920D2374920E236B920F2362
:1002B00062921023599211235092122347921323D2
:1002C0003E921423359215232C9216232392172342
:1002D0001A9218231192192308921A22FF921B16C0
:1002E000921C0AB89B1F9BFF9BFF9EFF8E9B0F9B40
:1002F000FF9BFF9EFF8E9B079BFF9BFF9EFF8E9B9E
:10030000039BFF9BFF9EFF8E9B019BFF9BFF9EFF1E
:100310008E9B009BFF9BFF9EFF8E9B009B7F9BFF06
:100320009EFF8E9B009B3F9BFF9EFF8E9B009B1F13
:100330009BFF9EFF8E9B009B0F9BFF9EFF8E9B0053
:100340009B079BFF9EFF8E9B009B039BFF9EFF8E48
:100350009B009B019BFF9EFF8E9B009B009BFF9E33
:10036000FF8E9B009B009B7F9EFF8E9B009B009BB4
:100370003F9EFF8E9B009B009B1F9EFF8E9B009BC2
:10038000009B0F9EFF8E9B009B009B079EFF8E9BFA
:10039000009B009B039EFF8E9B009B009B019EFF8A
:1003A0008E9B009B009B009EFF8E9B009B009B00F2
:1003B0009E7F8E9B009B009B009E3F8E9B009B0020
:1003C0009B009E1F8E9B009B009B009E0F8E9B00A0
:1003D0009B009B009E078E9B009B009B009E038EB4
:1003E0009B009B009B009E018E9B009B009B009EA0
:1003F000008E52BD06770F9D06933B19931D022276
:1004000071A1911E22719D0696FFBD057702940190
:10041000931D0222718ED242D1FFC1FEC2FC8E001A
:1004200000000000000000000000000000000000CC
:1004300000000000000000000000000000000000BC
:1004400000000000000000000000000000000000AC
:10045000000000000000000000000000000000009C
:00000001FF
